:1000000012C0189518951895189518951895189563
:100010001895189518951895189518951895189578
:100020001895189518958FED8DBFC0ECE0EC4E2E0D
:10003000DD275D2EEEE7F0E0A0E6B0E0A89584B7FE
:10004000082E877F84BF88E1992781BD91BD8827CD
:100050008D933197E9F75BD266248FEF81BB8EE1F8
:1000600087BBC09AC59AC69AC79AC29AC19AE6E84F
:10007000F0E080E494D258E0C895802D8AD2319681
:100080005A95D1F704C00C12120C20202020E6EA69
:10009000F0E080E584D258E0C895802D7AD2319680
:1000A0005A95D1F704C020201F1F1F1F202015D2F2
:1000B0008CE075D2E2E6F7E008D2E2E0F0E01ED292
:1000C0000CD2E2E7F7E001D206D2E8E7F7E0FDD193
:1000D000E3E0F0E013D201D2EAE0F0E0ABE61BD3BC
:1000E000E4E1F0E0ACE617D3EFE0F0E0A7E613D3ED
:1000F000EFE0F0E0A0E10FD3043608F00EC0EDD140
:10010000E8E8F7E0E2D1E7D1E2E6F7E0DED1C49833
:10011000C39885B7816285BF8895C298C0D1BFD189
:1001200080E08093600080E08093610081E08093B4
:10013000690000916900083010F009F01CC0A1E6C8
:100140000C9142E0F2D24C93AAD10091610040910F
:100150006000040FA1E60C93B09B04C081E0809383
:10016000600003C080E080936000A9E68C918F5FFF
:100170008C9308F4DECFC29A84E690E03CD2A4E6E9
:100180008C918F5F8C9300916400003408F001C063
:1001900014C080E08093640040916B000091610086
:1001A000041710F009F001C0C49A40916C0000914E
:1001B0006100041708F401C0C4988FE711E09CD1D6
:1001C000EAE9F7E082D1009161000A3008F003C04B
:1001D000EEE9F7E07AD1A8EAB0E0E1E6F0E03BD260
:1001E0006CD180E0D6D1E0EAF7E06FD18FE71AE07A
:1001F00083D1E4EAF7E069D1C49904C0EAEAF7E000
:1002000064D103C0EEEAF7E060D180916100809391
:100210006A0013D1BE98A8E69C9196FF04C0B69BD5
:100220000EC09F7B9C93B6990AC089E19F93992742
:10023000E2D19F91B69903C090649C9301D058CFAE
:10024000EFE0F0E0A7E667D28091670081508093ED
:100250006700EFE0F0E0A7E67BE74CD28091680012
:100260008F778093680039D1E2EBF7E02ED133D15C
:10027000E4ECF7E02AD1BD98A8E69C9195FF04C074
:10028000B59B0EC09F7D9C93B5990AC089E19F9351
:100290009927B1D19F91B59903C090629C934FD09B
:1002A000BF98A8E69C9194FF04C0B79B0EC09F7EA8
:1002B0009C93B7990AC089E19F9399279CD19F91FC
:1002C000B79903C090619C9379D0A8E68C9187FB85
:1002D0000EF401C02DC0EAE0F0E0ABE67BE70AD205
:1002E000E4E1F0E0ACE67BE705D2EAE0F0E0ABE683
:1002F00012D2E4E1F0E0ACE60ED240916C00009145
:100300006B00041708F414C0E8D0E6EDF7E0DDD088
:1003100000916B0041E0040FACE60C93E4E1F0E0E7
:10032000ACE67BE7E7D1E2E0F0E0E8D0D6D0089594
:10033000A8E68C9187FB0EF001C008959CCF80E069
:1003400080936B00CAD0B69906C08091680080681F
:10035000809368000895B59907C084E690E04BD17A
:10036000ABE68C918F5F8C938FE711E0C5D0E8EE00
:10037000F7E0ABD000916B000A3008F003C0EEE963
:10038000F7E0A3D0A8EAB0E0EBE6F0E064D195D0C6
:1003900080E0FFD0ECEEF7E098D080916B00809386
:1003A0006A004BD000916B00033610F009F001C0D9
:1003B00004C080E080936B0090D0C5CF80E0809334
:1003C0006C008BD0B69906C08091680080688093DD
:1003D00068000895B79907C084E690E00CD1ACE6B8
:1003E0008C918F5F8C938FE711E086D0E0EFF7E080
:1003F0006CD000916C000A3008F003C0EEE9F7E021
:1004000064D0A8EAB0E0ECE6F0E025D156D080E078
:10041000C0D0ECEEF7E059D080916C0080936A0078
:100420000CD000916C00033610F009F001C004C03C
:1004300080E080936C0051D0C5CF84E690E0DBD0A3
:100440008FEB11E059D000916A0042E07AD1A6E624
:100450000C938091660081508093660081E08093C8
:1004600067004091660000916700041710F009F0E2
:1004700010C000916600003110F009F001C001C009
:100480000DC082E086D0A7E68C918F5F8C9308F434
:10049000E8CF82E07ED0E4EFF7E017D00895969A97
:1004A000000000000000000000000000000000004C
:1004B00000000000000096980895A8EAB0E08D9131
:1004C000882311F066D0FBCF0895A4D0802D11F0C1
:1004D00060D0FBCF089580EC62C081E060D014D082
:1004E00080E85DC08FE7213039F08FEB223021F0BA
:1004F0008FE8233009F08FEC810F51C088EE93E034
:100500007AD03197D9F7089583E0992774C08AEF9C
:1005100090E071D08D9A8C9A8B9A8A9A899A889A4F
:10052000909885E090E067D0919895989498939AE8
:10053000929A919AEF93FF93E5E1F0E050D0FF910A
:10054000EF91919855D0919AEF93FF93E5E1F0E008
:1005500046D0FF91EF9191984BD0919AEF93FF93F2
:10056000E5E1F0E03CD0FF91EF91919841D0929875
:10057000919AEF93FF93E5E1F0E031D0FF91EF9195
:10058000919836D088E20BD08EE009D086E007D073
:100590000895909A829505D004D02AD00895909815
:1005A000F9CF859510F4929A01C09298859510F430
:1005B000939A01C09398859510F4949A01C09498E9
:1005C000859510F4959A01C09598919AEF93FF93B1
:1005D000E5E1F0E004D0FF91EF9191980895319713
:1005E000F1F70895689462F80895E89462F8089520
:1005F00081E090E000C0EF93FF93EE27E82BE92B1A
:1006000031F0EAEFF0E03197F1F70197D1F7FF9180
:10061000EF910895C895319600200895000F111F9D
:10062000221F331F089500951095209530950F5F78
:100630001F4F2F4F3F4F0895019110810EC0019120
:100640001191219130810BC00191108117FF05C0DC
:100650003FEF2FEF04C0008111272227332737FFF8
:1006600003C0E1DF8DE28D93CF93DF93CF92DF92D2
:10067000EF92AA24BB24CC24DD24EE2440E2CAE07D
:10068000DD2755E093E38881890F87FD9F7083FD07
:10069000907F891B89935A95A9F7C0DFAA1CBB1CC0
:1006A000CC1CDD1CEE1C4A9551F7E894EFE0FF27C7
:1006B00082910ED0EB30E0F71EF068948A2D0CD0BA
:1006C00088278D93EF90DF90CF90DF91CF910895A1
:1006D000982F829501D0892F8F70805D26F080330E
:1006E00009F4089568948D930895E199FECFEEBBC7
:1006F0003196089591E001C092E07B3751F47FB7C5
:10070000F894F3DF8D918DBBE29AE19A9A95C9F73F
:100710007FBF7727089591E001C092E0E6DFE09A7D
:100720008DB38D939A95D1F70895FF935527F8E0EF
:10073000469508F4500F57954795FA95D1F7FF91D4
:100740000895FF93881BF9E0001FFA9511F4FF91BB
:100750000895881F841B18F4840F8894F5CF08949B
:10076000F3CF5757572E4156522E344D472E434FF5
:100770004D0044454D4F000047534D3A3034302032
:100780003833323137390000212044454D4F204560
:1007900058504952454420210000543A000020009E
:1007A000432020004F55543A00004F4646004F4E1C
:1007B000200054313D4C4F57202D2054323D4849A4
:1007C000474800003C54313E20203C4F4B3E202007
:1007D0003C54323E00005432206D757374206265C3
:1007E000203E20543121000054313D0043200000C0
:0A07F00054323D00202020200000BC
:00000001FF
